:100000000C94C5020C9409030C9409030C94090385
:100010000C9409030C9409030C9409030C94090330
:100020000C9409030C9409030C94A7140C947915EF
:100030000C94DB220C9409030C9409030C9409031F
:100040000C9409030C946B030C9409030C9409039E
:100050000C9409030C9443230C9409030C94090396
:100060000C9409030C9409030C9409030C940903E0
:100070000C9409030C9409030C9409030C940903D0
:100080000C941C0B0C9409030C9409030C940903A5
:100090000C9409030C9409030C9409030C940903B0
:1000A0000C9409030C9409030C940903E615081633
:1000B000F6160816F6164D167016F616C516D8164C
:1000C000C219C219F119F119301A501AA61BA61B30
:1000D0005B1AA61B0B1B0B1B721B7B1BA61BA01BFF
:1000E000181B181B181B181B181B181B181B181B78
:1000F000181B181B181B181B181B181B181B181B68
:10010000281B361B3D1B441B4E1B07634236B79B07
:10011000D8A71A39685618AEBAAB558C1D3CB7CC67
:100120005763BD6DEDFD753EF6177231BF000000DF
:10013000803F08000000BE922449123EABAAAA2AC2
:10014000BECDCCCC4C3E00000080BEABAAAAAA3EDD
:1001500000000000BF000000803F00000000000819
:100160004178D3BB4387D1133D190E3CC3BD4282B6
:10017000AD2B3E68EC8276BED98FE1A93E4C80EF74
:10018000FFBE01C4FF7F3F00000000000000000030
:1001900000000000000000010204060A0F17202CD6
:1001A0003A4A5D71879DB3C7DAE9F5FCFFFCF5E9D2
:1001B000DAC7B39D87715D4A3A2C20170F0A0604EF
:1001C0000201000000000000000000000000F1A299
:1001D000F1A3F1A429002F003400330013001C0008
:1001E00009000A00060015000F002A002B00040079
:1001F0001200080018000C0007000B001700110087
:1002000016002800E100370014000D000E001B004E
:10021000050010001A0019001D003600E000E20081
:10022000E300032002202C002C0001200320E70023
:10023000E600E400000000000000000000000000F4
:1002400000000000000000000000000000000000AE
:10025000000000000000000000000000000000009E
:10026000000000000000000000000000000000008E
:10027000000000000000000000000000000000007E
:10028000000000000000000000000000000000006E
:100290000000000030141E001F002000210022007A
:1002A0002300240025002600270030023A003B00EE
:1002B0003C003D003E003F00400041004200430042
:1002C000440045000100010001000100010001009F
:1002D0000100010001000100010001000100010016
:1002E0000100010001000100010001000100010006
:1002F000010001002E021E021F022002221422020F
:10030000230224022414271427022D0001001F14A5
:100310003802640064022D1464143200250226029F
:100320002D02380001000100010001000100010060
:100330000100010025142614010001000100010044
:1003400001000100010001000100010001000100A5
:100350000100010001004A0052004D0001000100AF
:1003600001004A0052004D0001004C0001004F0006
:10037000510050004B0001004B00500051004F0055
:100380000100010001000100010001004E00010018
:100390004E000100AA00A9000100010001000100B7
:1003A0000100010001000100010001000100010045
:1003B000010001002803540068006500200050007F
:1003C0006C0061006E0063006B0020004B00650054
:1003D000790062006F0061007200640000002C036D
:1003E0004F007200740068006F006C0069006E00BE
:1003F00065006100720020004B006500790062001A
:100400006F006100720064007300000004030904BF
:1004100009026D00040100A0FA09040000010301B3
:100420000100092111010001223F00070581030895
:10043000000A090401000103010200092111010061
:1004400001224D000705820308000A090402000189
:100450000300000009211101000122360007058375
:100460000308000A09040300010300000009211128
:100470000100012239000705840310000112011058
:100480000100000008EDFE606001000102000105AE
:10049000010906A101050719E029E71500250195C5
:1004A0000875018102050819012905950575019155
:1004B000029501750391010507190029771500259B
:1004C00001957875018102C005010980A1018502AD
:1004D00016010026B7001A01002AB7007510950111
:1004E0008100C0050C0901A1018503160100269CAD
:1004F000021A01002A9C02751095018100C00501B5
:100500000902A1010901A100050919012905150028
:10051000250195057501810295017503810105018C
:10052000093009311581257F950275088106093842
:100530001581257F950175088106050C0A3802157D
:1005400081257F950175088106C0C005010906A1B6
:1005500001050719E029E7150025019508750181B6
:100560000295017508810105081901290595057590
:100570000191029501750391010507190029FF15E5
:100580000025FF950675088100C011241FBECFEF1E
:10059000DAE0DEBFCDBF04B603FE24C080911E03A7
:1005A00090911F03A0912003B09121038730904BBD
:1005B000A740B04BB9F410921E0310921F03109283
:1005C00020031092210314BE84B7877F84BF88E183
:1005D0000FB6F89480936000109260000FBEE0E0C8
:1005E000F8E3099511E0A0E0B1E0E0E1FAE502C02E
:1005F00005900D92A03CB107D9F713E0A0ECB1E053
:1006000001C01D92AE31B107E1F70E94ED110C94CB
:10061000062D0C9400000895089581E00895089532
:100620000C940C030C940D030C940F030E94D0281F
:1006300023E030E0281B3109220F2093C4010895E4
:10064000282F2F9880918000211108C0877F8093E8
:10065000800010928D0010928C001BC088608093E7
:100660008000233019F48FEF9FEF0FC083E090E0FC
:10067000821B9109880F991F2FEF3FEFA90102C03C
:10068000569547958A95E2F7CA0190938D0080931D
:100690008C000C9416030E94160384E08093C3011F
:1006A0001092C0010895279A2F988FEF9FEF909393
:1006B0008700809386008AE08093800089E18093A0
:1006C00081000E9439280C944B030E9453036E9AB8
:1006D000769A0C940B031F920F920FB60F9211246F
:1006E0002F933F938F939F93EF93FF93E091C101DB
:1006F000F091C201CF0101969093C2018093C10194
:100700000090C30102C0F695E7950A94E2F7EF73F3
:100710008091C001823019F4E03251F404C081307C
:1007200039F4EF3329F480916F008D7F80936F004F
:10073000F0E0E457FE4FE49121E031E0E29FC00198
:10074000E39F900D11240090C40102C096958795F7
:100750000A94E2F790938D0080938C00FF91EF91C3
:100760009F918F913F912F910F900FBE0F901F90EF
:10077000189581E008950C94B90308950C946503CD
:1007800080911502882309F448C08091D10190918D
:10079000D201009779F40E940D239093D2018093A7
:1007A000D1018091D30190E0009771F48091D40140
:1007B00090E00AC00E9419232091000130910101AC
:1007C0002817390740F329C00197880F991F880F10
:1007D000991FFC01EB52FE4F6081718182819381F0
:1007E0000E94820AE091D30184E0E89FF001112485
:1007F000EB52FE4F60817181828193814FE050E026
:100800000E943A0E8091D30190E001966091D4014C
:1008100070E00E94B62C8093D3010C9410031092C8
:1008200017020C944F0A0895089581E080931702EF
:100830000C941404089508958F929F92AF92BF92E2
:10084000EF92FF920F931F93CF93DF93CDB7DEB755
:10085000A3970FB6F894DEBF0FBECDBF7C01FC019D
:1008600000811181C8010E940A21B8010E9421065D
:100870008C01B7010E94BB03882309F4CCC100326C
:10088000F0E51F0741F4F7018281882309F458C07D
:100890000E949E0EC0C10132F0E51F0741F4F7012E
:1008A0008281882309F44CC00E94A70EB4C1023291
:1008B000F0E51F0751F4F7018281882309F440C055
:1008C0000E949A0E8111F0CFE3CF0332F0E51F07AB
:1008D00039F4F7018281882399F10E9415049BC1A4
:1008E0000432F0E51F0739F4F7018281882341F1D2
:1008F0000E940F0490C10532F0E51F0749F4F7018B
:1009000082818823E9F0809117028111F1CFE5CF30
:100910000632F0E51F0739F4F7018281882381F060
:100920000E94AE0E0AC00732F0E51F0749F4F70136
:100930008281882329F00E94B90E0E941B046BC19A
:1009400080911702811105C0F70182818111CFC00A
:1009500018C1003E110579F4F7018281882309F45A
:100960004DC00E944F0A81E080931602109215023A
:100970001092D40150C1023E110559F4F701828151
:100980008823E1F10E944F0A10921602109215027C
:1009900042C1033E110591F4F7018281882371F170
:1009A0000E944F0A1092160281E080931502109265
:1009B000D3011092D2011092D1012DC1023511053F
:1009C00059F4F7018281882309F425C1809100013F
:1009D000909101010A970DC00135110579F4F701D5
:1009E0008281882309F417C180910001909101014F
:1009F0000A9690930101809300010DC1409104017A
:100A000083E2EFE1F1E0DE01119601900D928A950B
:100A1000E1F7F701808121E030E02C0F3D1F280F26
:100A2000311DC9012091020130910301FC01E20F47
:100A3000F31F6081772767FD7095640F711D88270C
:100A400077FD8095982F0E94D82920E030E040E47F
:100A500051E40E943D294B015C01F701218184E0B2
:100A600090E0821B9109BC01882777FD8095982F23
:100A70000E94D8299B01AC01C501B4010E94D52870
:100A80009B01AC0160E070E080E090E40E944B2BA1
:100A900020E030E04CED50E40E94E82A4B015C017C
:100AA000F70182818823D1F04FE050E0C501B40105
:100AB0000E943A0E809116028823A1F08091D40101
:100AC00024E0829FF0011124EB52FE4F808291823C
:100AD000A282B3828F5F8093D40104C0C501B401A8
:100AE0000E94820A0F3F110508F02ECF94C080911A
:100AF000D00181111FC0043130E5130709F051C046
:100B00000E94BD0381E08093D0010E940D23909349
:100B1000CF018093CE011092C7011092C9011092AB
:100B2000C8011092CB011092CA011092CD0110920F
:100B3000CC0171C08091CE019091CF010E94192308
:100B4000883C910570F48091C701E82FF0E0EE0F2A
:100B5000FF1FE853FE4F118300838F5F8093C7010F
:100B60005AC0043880E5180721F00538104501F116
:100B70003AC0F7018281882341F01092C50182E0DA
:100B80001EC0043830E5130759F58091C501811165
:100B900006C086E20E94661886E20E942E1982E054
:100BA0001CC00438F0E51F0741F305381045D9F49F
:100BB000F7018281882331F01092C60180E20E9401
:100BC0007D1929C08091C601811106C087E20E946B
:100BD000661887E20E942E1980E20E9484191BC0C9
:100BE0000538104529F381E08093C5018093C60143
:100BF000C701A3960FB6F894DEBF0FBECDBFDF913D
:100C0000CF911F910F91FF90EF90BF90AF909F9069
:100C10008F900C94120380E0A3960FB6F894DEBF79
:100C20000FBECDBFDF91CF911F910F91FF90EF903D
:100C3000BF90AF909F908F90089580E090E00895CE
:100C400008959CE0799FF001112490E3899FE00DC5
:100C5000F11D1124E60FF11DEE0FFF1FEC52FE4FA8
:100C6000859194910895880F991FFC01E45BFF4FD3
:100C7000859194910895880F991FFC01E453FE4FCC
:100C80008591949108950F931F93CF93DF93EC0177
:100C9000811521E39207A0F5C11580E3D80708F07C
:100CA000D7C0C83ED105D8F4C03ED10508F007C270
:100CB000C83AD10578F4C53AD10508F06AC0C13008
:100CC000D10509F463C008F4F7C1C430D10508F0B8
:100CD000F6C1F2C1CB3BD10508F466C0EDC1C11528
:100CE00090E2D90708F0AFC0C11521E0D20708F0A3
:100CF000E6C1C03FD10508F4DFC18E0110651FC2F7
:100D0000C03880E5D80700F5C03790E5D90708F06E
:100D1000A3C0C11520E5D20709F4ACC050F4CE0140
:100D2000905480319F4008F0C7C1DF708E01106A77
:100D300006C2C13080E5D80709F4AEC0C43190E5E1
:100D4000D90708F4AFC0B8C1C33820E5D20709F409
:100D50008EC050F4C13890E5D90709F482C008F07C
:100D600083C000E011EDEBC1C03181E5D80708F484
:100D7000A3C1C11597E5D90708F436C1CE01905734
:100D80008115904108F098C1DF7093C101E010E037
:100D9000D6C1C53AD10509F494C1C63AD10509F0C6
:100DA00093C102E810E4CBC1C83AD10509F48FC160
:100DB000C93AD10509F48EC1CA3AD10509F48DC1E9
:100DC000CB3AD10509F48CC1CC3AD10509F48BC1D9
:100DD000CD3AD10509F48AC1C03BD10509F489C1D6
:100DE000CE3AD10509F488C1CF3AD10509F487C1BB
:100DF000C13BD10509F486C1C23BD10509F485C1C7
:100E0000C33BD10509F484C1C43BD10509F483C1B6
:100E1000C53BD10509F482C1C63BD10509F481C1A6
:100E2000C73BD10509F480C1C83BD10509F47FC196
:100E3000C93BD10509F47EC1CA3BD10509F47DC186
:100E400000E014E47CC1CE019F700E943B0678C193
:100E5000DD278E01106C73C1CF70DD278E01146DFC
:100E60006EC100E010ED6BC100E012ED68C100E062
:100E700013ED65C10E94111C0E944F0A0E941304C9
:100E80008FEF94E32CE0815090402040E1F700C0C8
:100E900000000E94682353C18091F2028160809318
:100EA000F2024DC10E94C923811102C00E94A523F4
:100EB0000E94DC2390E090931D0380931C03C230BA
:100EC00080E5D80721F480911C03816086C0C4307E
:100ED00090E5D90721F480911C0382607EC0C63062
:100EE00020E5D20721F480911C03846076C0C830CD
:100EF00080E5D80719F480911C0327C0CA3090E51B
:100F0000D90721F480911C03806167C0CC3020E5B3
:100F1000D20721F480911C0380625FC0CE3080E54F
:100F2000D80721F480911C03806457C0C03190E53C
:100F3000D90721F480911C0380684FC0C23120E59D
:100F4000D20729F480911C038460886046C0C330B6
:100F500080E5D80721F480911C038E7F3EC0C53008
:100F600090E5D90721F480911C038D7F36C0C730EE
:100F700020E5D20721F480911C038B7F2EC0C9305D
:100F800080E5D80719F480911C0326C0CB3090E58A
:100F9000D90721F480911C038F7E1FC0CD3020E53E
:100FA000D20721F480911C038F7D17C0CF3080E5DC
:100FB000D80721F480911C038F7B0FC0C13190E5CD
:100FC000D90721F480911C038F7707C0C331D04526
:100FD00031F480911C038B7F877F80931C03809169
:100FE0001C030E94E023ABC08D2F99278F70992797
:100FF00081309105D9F49E012370332702C0880FF8
:10100000991F2A95E2F79C688E0144E0000F111F9A
:101010004A95E1F700271370802B912B53E0CC0FFA
:10102000DD1F5A95E1F7C076DD272FC0823091058C
:1010300031F4DC2FCC278E01016F106A80C0833021
:10104000910569F4CE018370992701E010E002C098
:10105000000F111F8A95E2F7C8019C680FC0843009
:101060009105B9F4CE018370992701E010E002C028
:10107000000F111F8A95E2F7C8019A6823E0CC0F90
:10108000DD1F2A95E1F7C07ED7708C010C2B1D2B3C
:1010900056C08530910531F4DC2FCC278E01046FCA
:1010A000106A4DC0069709F04AC0CF71DD27DC2FCA
:1010B000CC278E01106243C000E010E040C08E01DA
:1010C0003EC001E810E43BC003E810E438C002EE83
:1010D00014E435C009EE14E432C00AEE14E42FC063
:1010E00005EB14E42CC006EB14E429C007EB14E470
:1010F00026C00CEC14E423C00DEC14E420C003E87B
:1011000015E41DC00AE815E41AC002E915E417C089
:1011100004E915E414C001E216E411C003E216E488
:101120000EC004E216E40BC005E216E408C006E2B5
:1011300016E405C007E216E402C00AE216E4C8019C
:10114000DF91CF911F910F9108959CE0799FF0015D
:10115000112490E3899FE00DF11D1124E60FF11D8C
:10116000EE0FFF1FEC52FE4F85919491803E91054A
:10117000E0F4803C910558F58133910509F46FC086
:1011800048F48932910509F463C08A32910509F463
:101190006DC072C089339105E9F082389105D1F0B4
:1011A0008533910509F44DC067C0833E910581F1F7
:1011B00038F4803E9105B9F0823E9105D9F05CC0CB
:1011C000863E910561F1873E9105A1F155C00E94CF
:1011D0003306089520911C0320FD02C021FF4CC05E
:1011E00080EE90E049C080911C0380FFF9CF89E335
:1011F00090E042C080911C0382FF0EC080911C03CE
:1012000084FF03C080E090E037C083EE90E034C0FC
:1012100080911C0382FFF2CF82EE90E02DC080917E
:101220001C0383FF0BC080911C0384FDEBCF87EE72
:1012300090E022C080911C0383FFF5CF86EE90E002
:101240001BC080911C0385FF07C089E290E014C099
:1012500080911C0385FFF9CF85E390E00DC080915C
:101260001C0386FF07C08AE290E006C080911C0341
:1012700086FFF9CF81E390E00E94430608950C9425
:101280001403E82FF0E0E25BFE4F8081E82FEF705F
:10129000F0E082958F7021E030E0A90102C0440F98
:1012A000551F8A95E2F740A308950F931F93CF939C
:1012B000DF9385B7806885BF85B7806885BFC3E049
:1012C000D0E001E010E0FE01E25BFE4F8081E82FFC
:1012D000EF70F0E021A182958F70A80102C0440F49
:1012E000551F8A95E2F7CA01822B81A38C2F0E9499
:1012F0004109219740F78BE090E061E070E0FC014C
:10130000EE5BFE4F2081E22FEF70F0E042A12295CC
:101310002F70DB0102C0AA0FBB1F2A95E2F79D01C7
:10132000242B22A3019758F7DF91CF911F910F91A2
:101330000C94BE03EF92FF920F931F93CF93DF9312
:1013400000E212E0C3E0EE24E394F12CD5E08C2F10
:101350000E9441098BE090E040E050E0FC01EE5B30
:10136000FE4F6081E62FEF70F0E020A130E0629543
:101370006F7002C0359527956A95E2F720FD09C088
:101380009701082E02C0220F331F0A94E2F7422B66
:10139000532B019718F7F801929182918F018417CE
:1013A000950721F051834083D09305018C2F0E9433
:1013B0004109C15060F68091050187FD2CC0815024
:1013C000809305018F3F39F08FE99FE00197F1F796
:1013D00000C0000020C080911E0290911F029093D7
:1013E00027028093260280911C0290911D02909307
:1013F00025028093240280911A0290911B029093FF
:1014000023028093220280911802909119029093F6
:101410002102809320020E94C00381E0DF91CF91DE
:101420001F910F91FF90EF900895E82FF0E0EE0FDD
:10143000FF1FE05EFD4F80819181089508950F9315
:101440001F93CF9308E212E0C0E0F80192918291DD
:101450008F010E948522C80FF2E000321F07A9F712
:101460008C2FCF911F910F9108950E94C923811154
:1014700002C00E94A5230E94EE23809307033E9A98
:10148000809171008D7F8093710082E08093900045
:101490008AE18093910081E080932A0208958091EF
:1014A0002A02811102C00E94350A10927A0210921B
:1014B0007902809171008D7F8093710080919000FE
:1014C0008F738093900010923C0210923B02109216
:1014D00073021092740210927502109276021092AA
:1014E000720210927102E1E5F2E0A1E4B2E0119221
:1014F0001192119211921D921D9282E0E137F8072C
:10150000B1F70895CF92DF92EF92FF920F931F935E
:10151000CF93DF9320913B02222309F484C06B0117
:101520007C0180912A02811102C00E94350A01E7E4
:1015300012E0C7E0D0E0A7019601F80192918291F4
:10154000729162918F010E943929811131C0FE018F
:10155000EE0FFF1FEE0FFF1FEF5AFD4F108211829B
:1015600012821382DE01AA0FBB1FAF5BBD4F119623
:101570001C921E92C730D105E9F021964481558115
:1015800066817781408351836283738314821582DD
:101590001682178212968D919C91139711969C93A7
:1015A0008E9313961C921E92129734961296E2CF47
:1015B000219708F68091790290917A02019797FD20
:1015C00005C090937A028093790204C010927A0247
:1015D000109279028091790290917A02209177029B
:1015E000309178022817390724F01092780210926F
:1015F0007702892BC1F4809171008D7F80937100F7
:10160000809190008F7380939000109273021092DB
:101610007402109275021092760210927202109269
:10162000710210923B02DF91CF911F910F91FF90B9
:10163000EF90DF90CF9008951F920F920FB60F9208
:1016400011244F925F926F927F928F929F92AF92EE
:10165000BF92CF92DF92EF92FF922F933F934F93DF
:101660005F936F937F938F939F93AF93BF93CF932A
:10167000DF93EF93FF9380913B02882309F49BC192
:10168000C0917902D0917A021C161D060CF093C10C
:1016900040902B0250902C0260902D0270902E02F0
:1016A00020E030E0A901C301B2010E94E42A18162B
:1016B0000CF065C0C130D10509F452C080917702A9
:1016C00090917802BE010E94B62C7C019093780222
:1016D0008093770280903D0290903E02A0903F025E
:1016E000B090400220E030E040E85FE3C501B40183
:1016F0000E94D52860933D0270933E0280933F0282
:1017000090934002F701EE0FFF1FEE0FFF1FEF5AFD
:10171000FD4FA301920160817181828193810E94BA
:101720003D2920E030E040E05EE30E94E82A9B0192
:10173000AC01C501B4010E94E42A18168CF4C7015B
:101740000196BE010E94B62C909378028093770296
:1017500010923D0210923E0210923F0210924002FF
:10176000E0917702F0917802EE0FFF1FEE0FFF1F5E
:10177000EF5AFD4F6081718182819381D0C0C0900A
:101780007302D0907402E0907502F090760220E02F
:1017900030E0A901C701B6010E94392921978823A9
:1017A00009F4A2C0FE01EE0FFF1FEE0FFF1FEF5A5C
:1017B000FD4F80809180A280B380A5019401C70174
:1017C000B6010E94392987FF31C0A501940160E06C
:1017D00070E08CED93EC0E943D2920E030E040E485
:1017E00051E40E943D2920E030E040E05FE30E94A8
:1017F000E82A9B01AC0160E070E080E090E40E9488
:101800004B2B9B01AC01C501B4010E94E82A9B014E
:10181000AC01C701B6010E94392987FF07C0A701A3
:10182000960160E070E08CED93E439C0A50194016D
:10183000C701B6010E94E42A18160CF055C0A50194
:10184000940160E070E08CED93E40E943D2920E07B
:1018500030E040E451E40E943D2920E030E040E0E7
:101860005FE30E94E82A9B01AC0160E070E080E049
:1018700090E40E944B2B9B01AC01C501B4010E9476
:10188000E82A9B01AC01C701B6010E94E42A1816A0
:101890005CF5A701960160E070E08CED93EC0E948E
:1018A0003D2920E030E040E451E40E943D2920E061
:1018B00030E040E05FE30E94E82A9B01AC0160E079
:1018C00070E080E090E40E944B2B9B01AC01C701CB
:1018D000B6010E94E82A60937302709374028093A9
:1018E00075029093760213C0FE01EE0FFF1FEE0FFC
:1018F000FF1FEF5AFD4F80819181A281B3818093B8
:10190000730290937402A0937502B0937602609173
:101910007302709174028091750290917602209109
:101920002802309129022F3F4FEF340731F02F5F0B
:101930003F4F30932902209328020E94C40E6B016E
:101940007C0120E034E244EF51E40E94392987FF12
:1019500008C086EFC82E88E2D82E84EFE82E81E4F6
:10196000F82E20E030E040E051E4C701B6010E94CB
:10197000E82A9B01AC0160E074E284E79BE40E94EA
:101980003D296B017C010E94AA2970939700609306
:101990009600209106013091070140910801509175
:1019A0000901C701B6010E94E82A0E94AA29709382
:1019B00099006093980080913C02882309F433C118
:1019C000C0903702D0903802E0903902F0903A028D
:1019D00020E030E0A901C701B6010E94E42A1816F0
:1019E000D4F580912802909129028F3F2FEF920722
:1019F00029F001969093290280932802C701B6012D
:101A00000E94C40E20E030E040E051E40E94E82A49
:101A10009B01AC0160E074E284E79BE40E943D29F5
:101A20006B017C010E94AA29709397006093960035
:101A30002091060130910701409108015091090160
:101A4000C701B6010E94E82A0E94AA297093990052
:101A50006093980008C01092970010929600109220
:101A600099001092980060913102709132026F5F7C
:101A70007F4F709332026093310220919600309133
:101A8000970080E090E0232BF1F0C0919600D09178
:101A900097000E94D6296B017C01BE0180E090E096
:101AA0000E94D6299B01AC016091330270913402EF
:101AB00080913502909136020E943D2920E03FEF4F
:101AC0004FE757E410C00E94D6296B017C0120E04B
:101AD00030EE4FEF54E46091330270913402809104
:101AE0003502909136020E94E82A9B01AC01C701A1
:101AF000B6010E94E42A87FD96C080912F028F5F75
:101B000080932F0290E02091030330910403821709
:101B10009307A0F080910E03882319F010922F02F2
:101B20000DC0809171008D7F809371008091900035
:101B30008F738093900010923C027DC080913002A0
:101B4000C0912F02811128C0C0900803D0900903D2
:101B5000E0900A03F0900B0320E030E0A901C701F8
:101B6000B6010E94E42A1816BCF481E0809330028A
:101B700010923702109238021092390210923A02F3
:101B8000C0923302D0923402E0923502F0923602D3
:101B9000C150C0932F0243C010923002109229020C
:101BA00010922802E0910503F091060348E0C49FDB
:101BB000E00DF11D112480819181A281B381809378
:101BC000370290933802A0933902B0933A0220E092
:101BD00030E040E85EE364817581868197810E94F0
:101BE000E82A6B017C0180910A01682F70E080E097
:101BF00090E00E94D62920E030E048EC52E40E94B8
:101C00003D299B01AC01C701B6010E94E82A6093FF
:101C1000330270933402809335029093360210920F
:101C20003202109231028091070380FD04C01092AD
:101C30003C0210923B02FF91EF91DF91CF91BF9157
:101C4000AF919F918F917F916F915F914F913F9154
:101C50002F91FF90EF90DF90CF90BF90AF909F902B
:101C60008F907F906F905F904F900F900FBE0F906E
:101C70001F901895CF92DF92EF92FF92CF93DF9350
:101C80006B017C01EA0180912A02811102C00E944D
:101C9000350A8091070380FF46C0809179029091B8
:101CA0007A0208970CF03FC0809171008D7F80937D
:101CB000710080913C0281110E944F0A81E0809363
:101CC0003B02109229021092280220E030E0A90184
:101CD000C701B6010E94E42A1816DCF4809179024B
:101CE00090917A02FC01EE0FFF1FEE0FFF1FEF5ADB
:101CF000FD4FC082D182E282F382FC01EE0FFF1F12
:101D0000EF5BFD4FD183C083019690937A0280935D
:101D100079028091710082608093710080919000BF
:101D2000806880939000DF91CF91FF90EF90DF90DB
:101D3000CF900895809107038170089580910703E3
:101D40008160809307030E94F2230C941A0480910F
:101D500007038E7F809307030C94F22380917B020C
:101D600090E0019666E070E00E94B62C80937B02C2
:101D7000089580917B0290E0019766E070E00E94F8
:101D8000B62C80937B0208958F929F92AF92BF9260
:101D9000CF92DF92EF92FF920F931F93CF93DF9337
:101DA0006B017C01C0912802D0912902BE0180E024
:101DB00090E00E94D6294B015C01A701960160E0EA
:101DC00070E08CE594E40E943D299B01AC01C501C3
:101DD000B4010E94E82A0E94AA2920917B022330A4
:101DE00009F473C028F4222351F02130E9F02CC10A
:101DF000243009F4A0C0253009F4E0C025C180E0FA
:101E000090E0A0E0BFE38093060190930701A093C8
:101E10000801B093090110922B0210922C0210922B
:101E20002D0210922E0210C110922B0210922C0241
:101E300010922D0210922E026431710540F46A3026
:101E4000710560F520E030E040E85EE32BC0693CBE
:101E5000710508F0AAC080E090E00E94D62920E039
:101E600030E040EA51E40E94D42820E030E044E32E
:101E700053E40E943D299B01AC010E94E82A20E026
:101E800030E040E05EE30E94E82A9B01AC0160E0A4
:101E900070E080E09EE30E94D42844C020E030E05F
:101EA00040E05FE3C701B6010E94E82A6B017C01B4
:101EB00080E090E0A0E0BEE38093060190930701EC
:101EC000A0930801B0930901BFC010922B02109299
:101ED0002C0210922D0210922E024AE0469F900191
:101EE000479F300D1124C90168EB7BE00E94A22CB2
:101EF000BC016C5D754077FF03C0719561957109F8
:101F0000882777FD8095982F0E94D8292EE333ECFF
:101F10004EE259E30E94E82A20E030E040EC5EE324
:101F20000E94D528609306017093070180930801F1
:101F30009093090189C010922B0210922C021092EA
:101F40002D0210922E02CE0183709927892BE1F089
:101F5000BE016170772780E090E00E94D62920E0E2
:101F600030E040E05EE30E94E82A20E030E040E418
:101F70005FE30E94D5286093060170930701809368
:101F80000801909309010CC080E090E0A0E0BFE35D
:101F90008093060190930701A0930801B093090173
:101FA000C770DD27CD2B09F04FC0109206011092AB
:101FB0000701109208011092090146C010922B02ED
:101FC00010922C0210922D0210922E0200E010E0CE
:101FD00020E03FE3009306011093070120930801DE
:101FE000309309016739710578F180E090E00E9433
:101FF000D62920E030E047E153E40E94D42820E0D5
:1020000030E04AE754E40E943D2920E030E048E413
:1020100052E40E94E82A20E030E040EA51E40E94C5
:102020001A2A0E94A529660F771F660F771FFB01EA
:10203000EE5AFE4F2081318142815381C701B601A2
:102040000E94E82A6B017C01C701B601DF91CF91A4
:102050001F910F91FF90EF90DF90CF90BF90AF90C6
:102060009F908F90089580918C020895CF93DF9375
:1020700000D01F92CDB7DEB79C018091130384304E
:1020800019F593E099833B832A839093E9008FEFBE
:102090009091E800815095FD06C095ED9A95F1F775
:1020A00000008111F5CF8091E80085FF0DC040E070
:1020B00050E063E070E0CE0101960E94971280919B
:1020C000E8008E778093E8000F900F900F90DF91DB
:1020D000CF910895CF93DF9300D01F92CDB7DEB795
:1020E00020911303243021F522E029839B838A83E6
:1020F00083E08093E9008FEF9091E800815095FD97
:1021000006C095ED9A95F1F700008111F5CF809109
:10211000E80085FF0DC040E050E063E070E0CE01D4
:1021200001960E9497128091E8008E778093E800D4
:102130000F900F900F90DF91CF910895209113038E
:102140002430F1F422E02093E9002FEF3091E800F1
:10215000215035FD06C035ED3A95F1F7000021110B
:10216000F5CF2091E80025FF0BC040E050E065E08E
:1021700070E00E9497128091E8008E778093E800CB
:102180000895CF93DF93EC0190911303943009F0FD
:1021900046C0809115018823D9F0809116018823CB
:1021A000B9F09093E9008FEF9091E800815095FD90
:1021B00006C095E19A95F1F700008111F5CF809165
:1021C000E80085FF2CC040E050E060E170E017C0FF
:1021D00081E08093E9008FEF9091E800815095FDB8
:1021E00006C095ED9A95F1F700008111F5CF809129
:1021F000E80085FF14C040E050E068E070E0CE01E8
:102200000E9497128091E8008E778093E80080E129
:10221000FE01ACE7B2E001900D928A95E1F7DF9103
:10222000CF91089580911203811109C00E942C144E
:102230000E9489148091E20084608093E2000895F6
:10224000109212030895089508950C94D02242E04C
:1022500061EC81E00E94A61342E061EC82E00E9402
:10226000A61342E061EC83E00E94A61342E161EC18
:1022700084E00C94A61380911503833009F455C0B3
:1022800030F4813071F0823009F48EC008958A30C4
:1022900009F47AC08B3009F460C0893009F09CC021
:1022A00020C080911403813A09F096C08091E80023
:1022B000877F8093E8008091180390911903892B00
:1022C00021F460E18CE792E003C060E080E090E000
:1022D00070E00E94E2128091E8008B778093E80022
:1022E000089580911403813209F076C0809118031B
:1022F00090911903009719F0039709F06DC0809130
:10230000E800877F8093E8008091E80082FD05C0A7
:10231000809113038111F8CF5FC08091F100809309
:102320008C028091E8008B7753C080911403813A2E
:1023300009F052C08091180390911903892B09F07C
:102340004BC08091E800877F8093E8008091E8008F
:1023500080FFFCCF8091150136C08091140381323B
:10236000D9F58091180390911903892BA9F58091D3
:10237000E800877F8093E8000E94DB1380911603BA
:10238000809315010C94111C80911403813221F566
:102390008091E800877F8093E8000E94DB138091A2
:1023A000170380938D02089580911403813AA1F45C
:1023B0008091E800877F8093E8008091E80080FFAB
:1023C000FCCF80918D028093F1008091E8008E77A0
:1023D0008093E8000C94DB13089584B7877F84BF53
:1023E00088E10FB6F89480936000109260000FBEF1
:1023F00090E080E80FB6F8948093610090936100BC
:102400000FBE0E947E170E942C140E948914809196
:10241000E20084608093E20078940E940F170E948B
:1024200080178BE091E00E942A178091130385307A
:1024300069F40E949122809111038823B1F30E94D4
:10244000BF22882391F30E948112EFCF0E94881748
:10245000ECCF292F332723303105C9F064F4213024
:10246000310581F02230310509F043C08DE690E05E
:1024700020E134E042C021323105F1F02232310551
:1024800041F137C082E190E02DE734E036C0992772
:102490008130910541F08230910541F0892B49F559
:1024A000ECE0F4E005C0EEEDF3E002C0E4EBF3E0B5
:1024B000849190E09F0121C06430D8F4E62FF0E0D1
:1024C000EE0FFF1FE255FE4F2081318189E090E041
:1024D00014C0643070F470E0FB01EE0FFF1FEA558A
:1024E000FE4F20813181FB01EE55FE4F808190E04F
:1024F00004C080E090E020E030E0FA0131832083E6
:10250000089580E189BD82E189BD09B400FEFDCF57
:102510008091D8008F7D8093D8008091E000826008
:102520008093E0008091E00081FDFCCF0895CF9280
:10253000DF92EF92FF920F931F93CF93DF93EC0103
:102540008B016A010E94FA13811133C0C114D104B6
:1025500039F0F60180819181081B190BC80FD91F32
:10256000E12CF12C0115110519F18091E80085FD90
:1025700016C08091E8008E778093E800C114D104E2
:1025800049F0F60180819181E80EF91EF182E08226
:1025900085E00FC00E94FA13882321F30AC08991B5
:1025A0008093F10001501109FFEFEF1AFF0ADACF13
:1025B00080E0DF91CF911F910F91FF90EF90DF901E
:1025C000CF90089520911A0330911B0326173707E7
:1025D00048F06115710539F42091E8002E772093B9
:1025E000E80001C0B90140E061157105A9F1209131
:1025F0001303222309F443C0253009F442C020917B
:10260000E80023FD40C02091E80022FD32C0209167
:10261000E80020FFE9CF4091F3002091F20030E084
:10262000342BFC01CF016115710559F028303105BB
:1026300040F481918093F100615071092F5F3F4F09
:10264000F1CF41E02830310509F040E02091E80069
:102650002E772093E800C8CF4111C9CF0AC08091DE
:102660001303882361F0853061F08091E80083FDD9
:102670000AC08091E80082FFF2CF80E0089582E0F6
:10268000089583E0089581E0089520911A03309120
:102690001B032617370748F06115710539F420919F
:1026A000E8002E772093E80001C0B901FC0120E08A
:1026B0006115710591F180911303882309F440C0DD
:1026C000853009F43FC08091E80083FD3DC08091D2
:1026D000E80082FD2FC08091E80080FFE9CF2091C3
:1026E000F3008091F20090E0922B6115710559F092
:1026F0008830910540F424912093F1003196615087
:1027000071090196F2CF21E0089709F020E080914D
:10271000E8008E778093E800CBCF2111CCCF0AC0A0
:1027200080911303882361F0853061F08091E80087
:1027300083FD0AC08091E80082FFF2CF80E0089517
:1027400082E0089583E0089581E00895982F9730FE
:1027500058F59093E900981739F07091EC002091AA
:10276000ED005091F00003C0242F762F50E021FFA0
:1027700019C03091EB003E7F3093EB003091ED00BB
:102780003D7F3093ED003091EB0031603093EB00F2
:102790007093EC002093ED005093F0002091EE0038
:1027A00027FF07C09F5FD3CF8F708093E90081E040
:1027B000089580E008958091140387FF11C08091EF
:1027C000E80082FD05C0809113038111F8CF11C08C
:1027D0008091E8008B770BC080911303882349F028
:1027E0008091E80080FFF8CF8091E8008E77809399
:1027F000E80008952091E4003091E50095E64091CD
:10280000EC00842F817040FF22C08091E80080FDA1
:102810001CC080911303882391F0853091F0809142
:10282000EB0085FD10C04091E4005091E500421797
:10283000530729F39A01915011F784E0089582E03B
:10284000089583E0089581E0089580E0089540911F
:10285000E80042FFDECF08950E949A140E94A2145D
:10286000E0EEF0E0808181608083E8EDF0E080813F
:102870008F77808319BCA7EDB0E08C918E7F8C930D
:1028800080818F7E80831092120308950F931F938F
:10289000CF93DF930E949A140E94A214C8EDD0E057
:1028A00088818F77888388818068888388818F7DFD
:1028B000888319BC1092130310920F031092110316
:1028C0001092100300EE10E0F80180818B7F80836E
:1028D00088818160888342E060E080E00E94A613E6
:1028E000E1EEF0E080818E7F8083E2EEF0E0808197
:1028F00081608083808188608083F80180818E7F01
:102900008083888180618883DF91CF911F910F91AF
:102910000895E8EDF0E080818F7E8083E7EDF0E0C0
:1029200080818160808384E082BF81E08093120394
:102930000C944614E8EDF0E080818E7F8083109245
:10294000E20008951092DA001092E10008951F92BB
:102950000F920FB60F9211242F933F934F935F93D3
:102960006F937F938F939F93AF93BF93EF93FF9357
:102970008091E10082FF0BC08091E20082FF07C0DE
:102980008091E1008B7F8093E1000E940E1780917F
:10299000DA0080FF1FC08091D80080FF1BC08091AB
:1029A000DA008E7F8093DA008091D90080FF0DC01D
:1029B00080E189BD82E189BD09B400FEFDCF81E0DF
:1029C000809313030E94121105C019BC10921303C7
:1029D0000E9420118091E10080FF19C08091E200E7
:1029E00080FF15C08091E2008E7F8093E20080918D
:1029F000E20080618093E2008091D8008062809341
:102A0000D80019BC85E0809313030E9424118091A3
:102A1000E10084FF30C08091E20084FF2CC080E19F
:102A200089BD82E189BD09B400FEFDCF8091D80047
:102A30008F7D8093D8008091E1008F7E8093E100AC
:102A40008091E2008F7E8093E2008091E2008160BD
:102A50008093E20080910F03882311F084E007C087
:102A60008091E30087FD02C081E001C083E0809394
:102A700013030E9425118091E10083FF29C08091FA
:102A8000E20083FF25C08091E100877F8093E10011
:102A900082E08093130310920F038091E1008E7FF8
:102AA0008093E1008091E2008E7F8093E20080912C
:102AB000E20080618093E20042E060E080E00E94FA
:102AC000A6138091F00088608093F0000E9423118B
:102AD000FF91EF91BF91AF919F918F917F916F91F6
:102AE0005F914F913F912F910F900FBE0F901F90CC
:102AF00018951F920F920FB60F9211242F933F93A8
:102B00004F935F936F937F938F939F93AF93BF93F5
:102B1000CF93DF93EF93FF93C091E900CF70809143
:102B2000EC00D82FD17080FDD0E81092E9008091A0
:102B3000F000877F8093F00078940E94BD1510927A
:102B4000E9008091F00088608093F000CD2BCF7079
:102B5000C093E900FF91EF91DF91CF91BF91AF91C9
:102B60009F918F917F916F915F914F913F912F91A5
:102B70000F900FBE0F901F9018951F93CF93DF9368
:102B8000CDB7DEB7AA970FB6F894DEBF0FBECDBFA4
:102B9000E4E1F3E088E08E0F9091F10091938E13C1
:102BA000FBCF0E943B118091E80083FF1FC1809101
:102BB000140390911503492F50E04A30510508F055
:102BC00015C1FA01EA5AFF4F0C94CA2C803881F0E3
:102BD000823809F00BC1809118038F708093E9004F
:102BE0008091EB0085FB882780F91092E90006C0F0
:102BF0008091100390911103911182609091E800EF
:102C0000977F9093E8008093F1001092F100C8C084
:102C1000282F2D7F09F0EAC0882319F0823061F057
:102C2000E5C080911603813009F0E0C0933009F0CF
:102C300080E0809311032BC080911603811127C07F
:102C4000809118038F7009F4D1C08093E90020911E
:102C5000EB0020FF1CC0933021F48091EB008062D8
:102C600014C09091EB0090619093EB0021E030E074
:102C7000A90102C0440F551F8A95E2F74093EA006C
:102C80001092EA008091EB0088608093EB00109234
:102C9000E9008091E800877F86C08111A7C010916C
:102CA00016031F778091E3008078812B8093E300E7
:102CB0008091E800877F8093E8000E94DB13809179
:102CC000E80080FFFCCF8091E30080688093E30000
:102CD000111102C082E001C083E08093130386C01B
:102CE0008058823008F082C08091160390911703BB
:102CF0008C3D53E0950779F583E08A838AE28983E6
:102D00004FB7F894DE01139620E03EE051E2E32F46
:102D1000F0E050935700E49120FF03C0E295EF707C
:102D20003F5FEF708E2F90E0EA3010F0C79601C041
:102D3000C0968D939D932F5F243149F74FBF8091AB
:102D4000E800877F8093E8006AE270E0CE01019698
:102D50000E94E21214C0AE014F5F5F4F60911803F2
:102D60000E942912BC01009709F440C09091E8002C
:102D7000977F9093E80089819A810E944513809102
:102D8000E8008B778093E80031C0803879F5809136
:102D9000E800877F8093E80080910F038093F10023
:102DA0008091E8008E778093E8000E94DB131EC0BC
:102DB00081111CC0909116039230C0F48091E800FC
:102DC000877F8093E80090930F030E94DB1380912C
:102DD0000F03811106C08091E30087FD02C081E0EE
:102DE00001C084E0809313030E9427118091E800C2
:102DF00083FF0AC08091E800877F8093E80080917C
:102E0000EB0080628093EB00AA960FB6F894DEBFC9
:102E10000FBECDBFDF91CF911F9108950895CF933D
:102E2000809113038823A1F0C091E900CF709091A5
:102E3000EC00892F817090FD80E8C82B1092E9008A
:102E40008091E80083FD0E94BD15CF70C093E9001A
:102E5000CF91089590939302809392020895E09108
:102E60009202F0919302309721F00190F081E02DD1
:102E7000099480E00895E0919202F09193023097D6
:102E800021F00280F381E02D09940895E0919202EF
:102E9000F0919302309721F00480F581E02D0994A0
:102EA000089520919002309191028217930771F05A
:102EB0009093910280939002E0919202F09193029C
:102EC000309721F00680F781E02D09940895209134
:102ED0008E0230918F028217930771F090938F02C8
:102EE00080938E02E0919202F0919302309721F04C
:102EF0000084F185E02D0994089508950C947D17C0
:102F00000E9404230E9455090E948A230C943928A8
:102F10005F926F927F928F929F92AF92BF92CF9269
:102F2000DF92EF92FF920F931F93CF93DF9300D026
:102F300000D01F92CDB7DEB70E949A099DE9C92E35
:102F400092E0D92E03E010E0AA24A394B12C502ED5
:102F5000802F0E94150A4C01F601729062906F0159
:102F60006826792661147104A1F40150110978F7DB
:102F70008FEF89838A831B820E940D238160782FC3
:102F80009D838C8349815A816B818D810E94381881
:102F900038C08091F20281FD0E941E0A2BE030E0D1
:102FA0007501022E02C0EE0CFF1C0A94E2F7C70165
:102FB00086219721892B09F129835A828E209F200F
:102FC00091E0892809F490E09B830E940D238160A1
:102FD000782F9D838C8349815A816B818D810E94DA
:102FE0003818000F111FF801EB56FD4F80819181B9
:102FF000E826F926F182E08204C02150310980F6EA
:10300000B4CF0E947125109194020E942F171817B7
:10301000D1F00E942F17809394020F900F900F9081
:103020000F900F90DF91CF911F910F91FF90EF9034
:10303000DF90CF90BF90AF909F908F907F906F90D8
:103040005F900C943F090F900F900F900F900F908E
:10305000DF91CF911F910F91FF90EF90DF90CF9074
:10306000BF90AF909F908F907F906F905F900895EA
:10307000CF93DF93CDB7DEB72B970FB6F894DEBFB3
:103080000FBECDBF4F83588769877A878B87DE0154
:10309000119686E0FD0111928A95E9F785E0FE011F
:1030A000379601900D928A95E1F749815A816B819B
:1030B0007C818D819E810E94AF1E2B960FB6F89465
:1030C000DEBF0FBECDBFDF91CF910895CF93882390
:1030D00009F4C2C0C82F823859F40E942F1781FD0D
:1030E000BBC089E30E9489210E94562289E30CC05B
:1030F000833879F40E942F1780FDAEC083E50E94CB
:1031000089210E94562283E50E94CB21CF910C9405
:103110005622843859F40E942F1782FD9DC087E4FF
:103120000E9489210E94562287E4EECF8CEF8C0FFB
:10313000813A48F48C2F0E94A12781118DC08C2FD9
:103140000E948921E3CF80E28C0F883048F4C77059
:1031500081E001C0880FCA95EAF70E940F22D6CFFE
:103160008BE58C0F833078F4C53A29F0C63A31F0FC
:1031700083E890E005C081E890E002C082E890E03A
:10318000CF910C94511788E58C0F833108F064C0FF
:10319000C83A39F1C93A41F1CA3A49F1CB3A51F149
:1031A000CC3A59F1CD3A61F1C03B69F1CE3A71F1B7
:1031B000CF3A79F1C13B81F1C23B89F1C33B91F137
:1031C000C43B99F1C53BA1F1C63BA9F1C73BB1F1A5
:1031D000C83BB9F1C93BC1F1CA3BC9F180E090E0FD
:1031E00038C082EE90E035C089EE90E032C08AEEC1
:1031F00090E02FC085EB90E02CC086EB90E029C0DA
:1032000087EB90E026C08CEC90E023C08DEC90E042
:1032100020C083E891E01DC08AE891E01AC082E9ED
:1032200091E017C084E991E014C081E292E011C0FE
:1032300083E292E00EC084E292E00BC085E292E06D
:1032400008C086E292E005C087E292E002C08AE20E
:1032500092E0CF910C946717CF910895882309F4D9
:103260004BC0823859F40E942F1781FF45C089E373
:103270000E9489210E94562289E30CC0833871F490
:103280000E942F1780FF38C083E50E9489210E9489
:10329000562283E50E94CB210C945622843859F49F
:1032A0000E942F1782FF28C087E40E9489210E9474
:1032B000562287E4EFCF9CEF980F913A58F390E2B3
:1032C000980F983050F4877091E001C0990F8A955B
:1032D000EAF7892F0E941522DFCF9BE5980F9330E4
:1032E00020F480E090E00C945117885A833120F448
:1032F00080E090E00C9467170895882321F00E94E5
:103300000F220C9456220895882321F00E94152242
:103310000C94562208957F928F929F92AF92BF9203
:10332000CF92DF92EF92FF920F931F93CF93DF9391
:103330001F92CDB7DEB77C01C62E772EFC0105812A
:1033400002950F70128111110E942C220E9482217D
:10335000882379F0112369F080E28C0D883048F0E1
:1033600082E00E946B210E94822191E0D82ED92612
:1033700001C0D12CE72DE295EF70F0E0E05AFF4F4D
:103380000C94CA2C872D807F072D0F70882311F095
:103390000295007F112389F0002309F499C180E28E
:1033A0008C0D883020F4802F0E940F2203C0802FC4
:1033B0000E941F220E9456228BC18C2D0E942E1922
:1033C000002309F4C3C180E28C0D883020F4802FE3
:1033D0000E94152203C0802F0E9425220E9456229F
:1033E000B5C1872D807F972D9F70803211F4892F72
:1033F00003C0892F8295807FCC2021F0F1E0CF1689
:10340000A1F01DC0112339F0002319F1013009F595
:103410000E943F229BC1002319F0013009F496C19C
:1034200089830E944222898110C1112321F0063034
:1034300008F08CC10EC0053008F088C106C1112308
:1034400059F0002331F0F701958190FF41C19F7041
:1034500095830E947D197AC1002309F4F6C03EC10C
:10346000872D86958695837090E0009719F00197D7
:1034700061F06CC1112321F08C2D972D937002C047
:1034800080E090E00E94511761C1112321F08C2D42
:10349000972D937002C080E090E00E94671756C19C
:1034A0008C2D112319F00E94792402C00E94E1247E
:1034B0000E9466254BC1872D837009F052C01111FF
:1034C00045C18C2D829586958770880F880F9C2D1D
:1034D0009F70892E912CA12CB12C082E04C0880C31
:1034E000991CAA1CBB1C0A94D2F7C4FE14C00FE09E
:1034F00010E020E030E0B901A80104C0440F551FDE
:10350000661F771F8A95D2F7CB01BA016095709537
:103510008095909503C060E070E0CB01272D269543
:103520002695237030E02230310569F023303105D3
:1035300089F0682979298A299B292130310571F080
:103540000E94F71F03C1682979298A299B290E94B3
:103550001320FCC00E94F71FC501B4010E94DB1FAD
:10356000F5C0112319F0872D817001C0869588233D
:1035700009F4ECC08C2D829586958770880F880F92
:103580009C2D9F70892E912CA12CB12C082E04C04B
:10359000880C991CAA1CBB1C0A94D2F7C4FE14C048
:1035A0000FE010E020E030E0B901A80104C0440FB2
:1035B000551F661F771F8A95D2F7CB01BA01609518
:1035C00070958095909503C060E070E0CB01272D49
:1035D000269526952370422F50E04230510569F020
:1035E0004330510589F0682979298A299B2941307E
:1035F000510571F00E94D120A9C0682979298A2932
:103600009B290E94ED20A2C00E94D120C501B401D7
:103610000E94B5209BC08C2D90E0FC01E05EF1097A
:10362000E531F10508F050C0E059FF4F0C94CA2C69
:103630000C2D0F70872D8F71112321F00E944E20C9
:10364000802F07CF0E946F20802F0E9484197EC098
:10365000112341F0053008F079C0872D8F710E9449
:10366000942074C0063008F071C0F7CF112339F0F0
:10367000872D8F710E944E2069C01123C9F3872DB9
:103680008F710E946F2062C0112329F0872D8F71E6
:103690000E9439205BC00E942F2058C0112351F096
:1036A000172D1F71812F0E944E2063E0812F0E94F1
:1036B00062214CC081E00E946B21023008F446C0B8
:1036C00082E00E946B2142C0112331F0002381F27D
:1036D0008C2D0E9466183AC0002389F28C2D0E941E
:1036E0002E1934C0472D4F706C2DC7010E941D0646
:1036F0000E94531F2BC0111129C0472D4F7050E05D
:1037000042305105B9F04CF44115510581F041307A
:103710005105E1F40E94612819C04330510569F058
:103720004430510599F48C2D0E94B3280FC00E949B
:103730004A280CC00E947D2809C00E94902806C01B
:10374000472D4F706C2DC7010E942006DD20F9F037
:103750000E945E2180FD1BC0F70112820E94582149
:103760000E944E20C7010E94D61B0E9458210F9034
:10377000DF91CF911F910F91FF90EF90DF90CF904D
:10378000BF90AF909F908F907F900C946F200F9080
:10379000DF91CF911F910F91FF90EF90DF90CF902D
:1037A000BF90AF909F908F907F9008950F931F933D
:1037B000CF93DF93EC01888199812B813C81232B6E
:1037C000B9F09F3F11F48F3F99F0CE010E941C0485
:1037D000882371F0688179818A810E9454218C014B
:1037E0000E9409210E94D01FB801CE010E948B19AE
:1037F000DF91CF911F910F9108950E942C220E947A
:103800003C220E9401220E9456220E9417260E94FA
:10381000662580E090E00E94511780E090E00C94D3
:1038200067170E941C220C94FD1B0E944921292F1E
:1038300022952F7030E02C3031054CF42A303105C0
:103840006CF42250310922303105A8F407C02C3025
:10385000310569F02F30310551F00DC0803F69F01E
:1038600018F4803E40F409C0843F29F406C093FB5D
:10387000882780F9089580E0089581E00895CF9326
:10388000DF9300D000D01F92CDB7DEB70F900F901E
:103890000F900F900F90DF91CF910895CF93DF930A
:1038A00000D000D000D0CDB7DEB726960FB6F89482
:1038B000DEBF0FBECDBFDF91CF9108951F93CF9391
:1038C000DF93C0919D0216E080919E02C81799F087
:1038D000D0E01C9FF0011D9FF00D1124E156FD4F1B
:1038E0004081518162817381848195810E944E1C47
:1038F0002196C770E9CFDF91CF911F910895409134
:10390000CF025091D0026091D1027091D202809189
:10391000D3029091D4020C944E1C8091D4028295D3
:103920008F7009F054C08091D102882309F44FC0F0
:1039300080919D02A0919E026091CF027091D00271
:103940004091D2025091D302B6E08A1709F43FC0E9
:1039500090E041155105C1F17F3F11F46F3FA1F196
:10396000B89FF001B99FF00D1124E156FD4F218160
:1039700072132AC02081621327C02281211124C022
:10398000238134812417350710F421503109241B79
:10399000350B283C3105C0F42091D4022F702061F2
:1039A0002093D40226E0289FF001299FF00D1124D6
:1039B000EC55FD4F80818F70806180838FEC92E0A9
:1039C0000E94D61B0C945E1C01968770BECF089592
:1039D000CF92DF92EF92FF920F931F93CF93DF93DB
:1039E000CDB7DEB762970FB6F894DEBF0FBECDBF7E
:1039F0008C0185E0F801DE011D9601900D928A95FB
:103A0000E1F7D8014C9111965C91119712966C9147
:103A100012971396CD90DC9014973091CF0270914D
:103A2000D0028091D2029091D302009709F46BC129
:103A30007F3F19F43F3F09F466C1E090D102EE20C8
:103A400009F4C0C02091D402C816D90628F0F601A6
:103A5000E81BF90BCF0104C0809590958C0D9D1D3E
:103A6000FF24F394883C910578F0F12C207F09F035
:103A7000C6C07C2DD98AC88A89890E943F1C8FECD8
:103A800092E00E94D61BB1C0822F807F09F046C011
:103A9000751314C0341312C0611110C02F7020614F
:103AA0002093D4020E947F1C8FEC92E00E94D61BD0
:103AB0008091D402D80115968C932EC0CD2819F18F
:103AC0005F3F11F44F3FF9F0F62E61111CC0809159
:103AD0009D0220919E0236E0821709F45AC090E0C0
:103AE000389FF001399FF00D1124E156FD4F71818F
:103AF000571306C07081471303C07281711103C050
:103B000001968770E9CFF62E662309F418C18091DB
:103B1000D40281608093D402F12C11C1751308C0C6
:103B2000341306C0611104C08091D402D801C3C00F
:103B30004D875E878D859E856A8B0E94151C6A89DC
:103B40008823E1F16623D1F12091D402822F82955E
:103B50008F7090E0029774F08091CF029091D00224
:103B600098878F831986DB86CA862C87CE010796B5
:103B70000E94D61B86E0F801AFECB2E001900D92F6
:103B80008A95E1F70E948D1C0E947F1CFF24F3940C
:103B9000D6C04D875E878D859E850E944921292F3D
:103BA00022952F7030E0223031050CF0BCC09F70A0
:103BB00009F0B6C0805E883008F4C1C0C8010E9418
:103BC000D61BE4CFC816D90608F453C0F601E81B8B
:103BD000F90BCF01883C910508F450C0F12C7C2DE5
:103BE000D98AC88A89890E943F1CEFECF2E086E0FE
:103BF000DF011D928A95E9F70E947F1CA0C0751312
:103C000014C0341312C0611110C08091D402F801A5
:103C10008583C8010E94D61B86E0EFECF2E0DF014D
:103C20001D928A95E9F7FE2C8AC04D875E878D85A7
:103C30009E856A8B0E94151C6A89882309F4BECF71
:103C4000662309F4BBCF2091D402822F82958F7016
:103C500090E002970CF48ECF8091CF029091D00229
:103C60009A8389831B82DD82CC822E83CE010196CA
:103C70007FCF809590958C0D9D1DACCFF62E662341
:103C800009F49CCF75132EC034132CC02091D4029C
:103C900020FD1FC0822F82958F70D9F0D801159614
:103CA0002C9315978F3049F08F5F982F9295907FC6
:103CB000822F8F70892B15968C93C8010E94D61B7A
:103CC00086E0F801AFECB2E001900D928A95E1F741
:103CD00093CF86E0F801AFECB2E001900D928A95A7
:103CE000E1F72DC04D875E878D859E850E94151C4E
:103CF000811140CF8091D40281608093D402C801A9
:103D00000E94D61B1CC0662309F458CF4D875E87DE
:103D10008D859E850E94151C882309F44FCF2ACFDC
:103D2000811148CF0CC0243031050CF047CF9F7073
:103D300009F440CFF8019581907F09F03BCF8F2D9A
:103D400062960FB6F894DEBF0FBECDBFDF91CF9164
:103D50001F910F91FF90EF90DF90CF9008951F93E8
:103D6000CF93DF93CDB7DEB72C970FB6F894DEBFB5
:103D70000FBECDBF4F83588769877A878B879C8713
:103D8000CE0107960E94E81C882369F08F819885F0
:103D90002A853B85232BF1F19F3F09F063C08F3FBC
:103DA00009F060C037C086E0FE013796DE0111964B
:103DB00001900D928A95E1F76F817885EA85FB8500
:103DC000309741F17F3F11F46F3F21F120919E0226
:103DD00030E0C90101968770992740919D0250E01B
:103DE0008417950709F447C069837A83FD83EC83C0
:103DF00096E0929FD001939FB00D1124A156BD4F24
:103E0000FE01319601900D929A95E1F780939E0202
:103E10000E945E1C16E080919D0290919E0289177F
:103E2000C1F1189FC001112481569D4F0E94E81CCA
:103E3000882379F1E0919D021E9FF0011124E15643
:103E4000FD4F4081518162817381848195810E94FF
:103E50004E1C80919D0290E0019687709927809377
:103E60009D02D9CF4F81588569857A858B859C8540
:103E70000E944E1CCFCF0E94111C10929E021092E5
:103E80009D02EFECF2E086E0DF011D928A95E9F7F2
:103E9000C1CF2C960FB6F894DEBF0FBECDBFDF9119
:103EA000CF911F910895EF92FF920F931F93CF939D
:103EB000DF938C01009709F46CC0F12CEE24E3949D
:103EC000E8012196F8018491843740F4843008F0A9
:103ED00051C0813081F0823019F15BC0853709F41F
:103EE00044C0A8F19CE7980F903708F052C08F7734
:103EF0000E942E1941C00E5F1F4FFE01C49180E247
:103F00008C0F883048F4C7708E2D01C0880FCA9579
:103F1000EAF70E942F2214C08C2F0E9466182DC031
:103F20000E5F1F4FFE01C49180E28C0F883058F461
:103F3000C7708E2D01C0880FCA95EAF70E943522FE
:103F40000E9456221AC08C2F0E942E1916C00E5F96
:103F50001F4FFE01C491CC2381F08FE99FE00197B0
:103F6000F1F700C00000C150F6CF0E5F1F4FFE01F9
:103F7000F49003C00E9466188E018F2D882309F4E7
:103F80009FCFEFE9FFE03197F1F700C000008150CB
:103F9000F5CFDF91CF911F910F91FF90EF90089592
:103FA00008956093D9027093DA028093DB029093B4
:103FB000DC020C94FD1B0F931F930091D90210910A
:103FC000DA022091DB023091DC02DC01CB01802B94
:103FD000912BA22BB32B8093D9029093DA02A0935A
:103FE000DB02B093DC021F910F910C94FD1B0F9329
:103FF0001F930091D9021091DA022091DB023091D7
:10400000DC02DC01CB0180239123A223B323809324
:10401000D9029093DA02A093DB02B093DC021F91E5
:104020000F910C94FD1B0F931F930091D9021091D7
:10403000DA022091DB023091DC02DC01CB01802727
:104040009127A227B3278093D9029093DA02A093F5
:10405000DB02B093DC021F910F910C94FD1B1092B8
:10406000D5021092D6021092D7021092D8020C9468
:10407000FD1B41E050E060E070E004C0440F551FBC
:10408000661F771F8A95D2F74093D5025093D602C8
:104090006093D7027093D8020C94FD1B41E050E06E
:1040A00060E070E004C0440F551F661F771F8A95BB
:1040B000D2F78091D5029091D602A091D702B0910B
:1040C000D802482B592B6A2B7B2B4093D502509357
:1040D000D6026093D7027093D8020C94FD1B41E086
:1040E00050E060E070E004C0440F551F661F771F6A
:1040F0008A95D2F740955095609570958091D5023C
:104100009091D602A091D702B091D80248235923AA
:104110006A237B234093D5025093D6026093D70243
:104120007093D8020C94FD1B41E050E060E070E019
:1041300004C0440F551F661F771F8A95D2F78091E0
:10414000D5029091D602A091D702B091D80248270B
:1041500059276A277B274093D5025093D602609354
:10416000D7027093D8020C94FD1B0F931F930091FC
:10417000D5021091D6022091D7023091D802DC01ED
:10418000CB01802B912BA22BB32B8093D502909344
:10419000D602A093D702B093D8021F910F910C942E
:1041A000FD1B0F931F930091D5021091D602209111
:1041B000D7023091D802DC01CB0180239123A223C6
:1041C000B3238093D5029093D602A093D702B093E5
:1041D000D8021F910F910C94FD1B0F931F93009118
:1041E000D5021091D6022091D7023091D802DC017D
:1041F000CB0180279127A227B3278093D5029093E4
:10420000D602A093D702B093D8021F910F910C94BD
:10421000FD1B0895CF92DF92EF92FF920F931F93B1
:10422000CF93DF938C01C090D902D090DA02E09056
:10423000DB02F090DC028091D5029091D602A09131
:10424000D702B091D802C82AD92AEA2AFB2ACFE19C
:10425000D0E0D701C6010C2E04C0B695A79597955E
:1042600087950A94D2F780FF06C0B8018C2F0E9470
:10427000A508019721F4219760F780E001C08C2FF9
:10428000DF91CF911F910F91FF90EF90DF90CF9032
:104290000895CF93DF93EC010E940A21BE010E9492
:1042A000A508DF91CF910895CB010E94492108957F
:1042B0008091DD0285958595859508958091DD0233
:1042C0008770089598E0899F90011124262B2093F0
:1042D000DD020C944E202091DD0280958223809394
:1042E000DD02982F977069F430E0482F552747FD7D
:1042F00050952417350729F08595859585950C945B
:104300006F2008959091DD02977081E009F480E0BC
:10431000089590911501992321F090911601911122
:1043200009C02091170130911801F90132969FEFD1
:1043300040E01FC0982F9695969596959F3050F522
:10434000E0911701F0911801E90FF11D877021E04C
:1043500030E0A90102C0440F551F8A95E2F7CA0157
:104360009181892B818308959F3F39F04F5F4E30B3
:1043700041F051915813F8CF0DC05111F7CF942F40
:10438000F5CF9F3F39F0F901E90FF11D97FDFA953F
:1043900082830895089590911501992321F09091B9
:1043A0001601911109C02091170130911801F901EE
:1043B0003296205F3F4F1FC0982F96959695969501
:1043C0009F30F0F4E0911701F0911801E90FF11D11
:1043D000877021E030E0A90102C0440F551F8A9583
:1043E000E2F7CA01809591818923818308953196EE
:1043F000E217F30729F090819813F9CF1082F7CFD5
:10440000089581E090E0E0911701F0911801E80F24
:10441000F91F1082019680319105A9F708959091B6
:10442000F102892B8093F102089580959091F10219
:1044300089238093F10208951092F10208959091DA
:10444000F002892B8093F002089580959091F002FC
:1044500089238093F00208951092F00208959091BC
:10446000EF02892B8093EF02089580959091EF02DF
:1044700089238093EF0208951092EF0208958093AC
:10448000DE0208951092DE02089580911701909146
:104490001801FC0131969C01205F3F4F80E0919113
:1044A00091118F5FE217F307D1F70895E09117019B
:1044B000F09118018091F1028083E0911701F09151
:1044C000180190818091F002892B8083E09117017F
:1044D000F091180190818091EF02892B8083809167
:1044E000DE02882361F0E0911701F09118019081BC
:1044F000892B80830E94452281111092DE028091D7
:104500001701909118010C943B1720E0009739F0A7
:10451000AC0141505109842395232F5FF7CF822F9F
:10452000089580911303843039F11092F30220E44E
:1045300088E190E00FB6F894A895809360000FBED4
:104540002093600080E00E94200380E00E943F09E9
:1045500083B7817F846083BF83B7816083BF789492
:10456000889583B78E7F83BF88E10FB6F8948093D8
:104570006000109260000FBE08950895089580E0D5
:104580000E9420030E94BD220E949A090E94BE221E
:104590000E941F0A91E0811101C090E0892F0895C7
:1045A0000E94111C80E00E9420030E9439280E9472
:1045B0002F170C943F091F920F920FB60F921124E0
:1045C0008F939F93AF93BF938091F302811113C098
:1045D0008091F4029091F502A091F602B091F70259
:1045E0004196A11DB11D8093F4029093F502A09312
:1045F000F602B093F702BF91AF919F918F910F9008
:104600000FBE0F901F90189582E084BD93E095BD7A
:104610009AEF97BD80936E0008952FB7F89480911C
:10462000F4029091F502A091F602B091F7022FBF2B
:104630000895CF92DF92EF92FF920F931F932FB7BF
:10464000F8944091F4025091F5026091F602709155
:10465000F7022FBF6A017B01EE24FF248C0120E0CA
:1046600030E0C016D106E206F30610F441505109BD
:104670009A01281B390BC9011F910F91FF90EF90F0
:10468000DF90CF9008951F920F920FB60F921124D2
:104690008F939F93AF93BF938091F4029091F50213
:1046A000A091F602B091F7020196A11DB11D809371
:1046B000F4029093F502A093F602B093F702BF9133
:1046C000AF919F918F910F900FBE0F901F901895F3
:1046D0000E942C14F8942FEF87EA91E62150804035
:1046E0009040E1F700C0000087E090EBDC01809390
:1046F0001E0390931F03A0932003B09321039CE01B
:1047000088E10FB6F894A895809360000FBE90934F
:104710006000FFCF0E94C923811102C00E94A5231F
:104720000E94D4238093F2020E94DC2380931C0316
:1047300087FB882780F9809316010E94D823682F71
:1047400070E080E090E00C94D11F6DEE7EEF80E091
:1047500090E00E94F02C60E082E090E00E94DE2C6D
:1047600060E083E090E00E94DE2C60E084E090E076
:104770000E94DE2C60E085E090E00E94DE2C60E08C
:1047800086E090E00E94DE2C6FEF87E090E00C94D2
:10479000DE2C80E090E00E94D82C21E08D3E9E4FE0
:1047A00009F020E0822F089582E090E00C94D02C54
:1047B00083E090E00C94D02C84E090E00C94D02C1A
:1047C000682F84E090E00C94DE2C86E090E00C945E
:1047D000D02C682F86E090E00C94DE2C87E090E0EF
:1047E0000C94D02C682F87E090E00C94DE2C809104
:1047F000FA0280FF0BC060911C0185E0689FB00148
:10480000112475956795759567952BC081FF09C033
:1048100060911C0185E0689FB00111247595679532
:1048200020C082FF07C060911C0185E0689FB00135
:10483000112417C09091FB029923D1F060911B01C4
:10484000961788F720911C0185E0289F900111247C
:10485000929FA001939F500D112470E0CA010E9405
:10486000B62C6038710540F46115710539F002C04D
:1048700065E070E0862F08958FE7089581E0089540
:104880008091FA0280FF08C060911A0170E075956E
:1048900067957595679521C081FF06C060911A01E3
:1048A00070E07595679519C082FF04C060911A0188
:1048B00070E010C09091FB029923C1F06091190142
:1048C0009617A0F780911A01899FC001112470E00A
:1048D0000E94B62C6038710528F46115710521F02D
:1048E000862F08958FE7089581E0089561E070E0D4
:1048F000F4CF803F21F40E94F723819504C0813FCB
:1049000029F40E94F7238093FE020895823F21F448
:104910000E94F723819504C0833F29F40E94F72366
:104920008093FD020895893F19F40E94402405C038
:104930008A3F31F40E94402481958093FF020895BC
:104940008B3F21F40E944024819504C08C3F29F4C0
:104950000E944024809300030895843F21F48091B5
:10496000FC02816017C0853F21F48091FC028260C7
:1049700011C0863F21F48091FC0284600BC0873F08
:1049800021F48091FC02886005C0883F31F4809159
:10499000FC0280618093FC0208958D3F21F4809198
:1049A000FA0281600BC08E3F21F48091FA0282608E
:1049B00005C08F3F29F48091FA0284608093FA0247
:1049C0000895803F39F48091FE0287FF6CC01092F9
:1049D000FE0269C0813F29F48091FE021816BCF3E3
:1049E00062C09091FD02823F29F497FF5CC0109253
:1049F000FD0259C0833F19F41916CCF354C0893F06
:104A000041F48091FF0218160CF04DC01092FF0285
:104A10004AC08A3F29F48091FF0287FF44C0F6CF45
:104A20008B3F39F48091000387FF3DC01092000353
:104A30003AC08C3F29F4809100031816BCF333C0B0
:104A4000843F21F48091FC028E7F17C0853F21F4C2
:104A50008091FC028D7F11C0863F21F48091FC0281
:104A60008B7F0BC0873F21F48091FC02877F05C0BC
:104A7000883F31F48091FC028F7E8093FC0213C04A
:104A80008D3F21F48091FA028E7F0BC08E3F21F47E
:104A90008091FA028D7F05C08F3F29F48091FA0240
:104AA0008B7F8093FA028091FD0281110EC080916C
:104AB000FE0281110AC08091FF02811106C080911F
:104AC0000003811102C01092FB0208958CEF92E066
:104AD0000E9446170E940D239093F9028093F802DA
:104AE00008951F93CF93DF938091F8029091F9027C
:104AF0000E941923AC019091FB02992321F020918F
:104B00001D0130E006C020911E018AE0289F90011F
:104B100011244217530708F486C08091FD02C0910A
:104B2000FE02D091FF0210910003811107C0C11154
:104B300076C0D11174C0111172C075C09F3F19F0B9
:104B40009F5F9093FB02181624F40E94F723809332
:104B5000FD028091FD0287FF05C00E94F723819529
:104B60008093FD021C1624F40E94F7238093FE021A
:104B70008091FE0287FF05C00E94F72381958093F4
:104B8000FE026091FD02662339F1C091FE02CC2342
:104B900019F1772767FD7095872F972F0E94D829E5
:104BA00023E333E343E35FE30E94E82A0E94A5295D
:104BB0006093FD026C2F772767FD7095872F972FE5
:104BC0000E94D82923E333E343E35FE30E94E82A0A
:104BD0000E94A5296093FE021D1624F40E94402421
:104BE0008093FF028091FF0287FF05C00E9440244E
:104BF00081958093FF02111624F40E944024809333
:104C000000038091000387FF05C00E944024819526
:104C100080930003DF91CF911F910C9466259F3FF5
:104C200009F08ECF96CFDF91CF911F910895ECEFD1
:104C3000F2E085E0DF011D928A95E9F71092FB0210
:104C40001092FA020895833081F128F4813059F0EE
:104C50008230D1F00895853009F449C0B8F186302A
:104C600009F456C0089580911E01262F30E0280FC8
:104C7000311D2F3F310524F4680F60931E01089504
:104C80008FEF80931E01089580911D01262F30E043
:104C9000280F311D2F3F310524F4680F60931D014B
:104CA00008958FEF80931D01089580911C01262F98
:104CB00030E0280F311D2F3F310524F4680F609339
:104CC0001C0108958FEF80931C01089580911B01B2
:104CD000262F30E0280F311D2F3F310524F4680FB7
:104CE00060931B0108958FEF80931B0108958091BD
:104CF0001A01262F30E0280F311D2F3F310524F4F3
:104D0000680F60931A0108958FEF80931A01089538
:104D100080911901262F30E0280F311D2F3F3105DA
:104D200024F4680F6093190108958FEF809319019F
:104D30000895833011F128F4813049F0823091F0E8
:104D40000895853081F120F18630C1F10895809178
:104D50001E01681720F4861B80931E01089510928F
:104D60001E01089580911D01681720F4861B809311
:104D70001D01089510921D01089580911C0168176E
:104D800020F4861B80931C01089510921C01089545
:104D900080911B01681720F4861B80931B010895E6
:104DA00010921B01089580911A01681720F4861B48
:104DB00080931A01089510921A01089580911901A3
:104DC000681720F4861B8093190108951092190129
:104DD00008950F931F93873208F048C08E3108F072
:104DE0008DC0803109F477C008F5873009F461C0BF
:104DF00068F4863009F09DC08091F202817F8E7F39
:104E00008093F20281E08093020394C08B3009F416
:104E100089C08E3009F08DC08091F20282FB22277A
:104E200020F991E0922790FB82F95EC0863109F467
:104E300079C060F4813109F07CC00E94111C90910E
:104E4000160181E08927809316016CC0893109F42D
:104E500069C08B3109F06DC08091F20281FB22277D
:104E600020F991E0922790FB81F93EC0883309F444
:104E700059C050F4893209F457C0853309F454C03D
:104E8000873209F451C055C0833409F44DC028F469
:104E90008A3308F44EC0895332C0883409F049C0BF
:104EA0000E94111C0E944F0A0E9413040E94682352
:104EB00039C09091F202892F8095817080FB90F922
:104EC00029F0966098609093F20234C0997F977FA2
:104ED0009093F20227C08091F20283FB222720F9EF
:104EE00091E0922790FB83F98093F2029923D1F00D
:104EF0008091F20281608093F20214C08D5141E0F2
:104F000050E060E070E08A019B0104C0000F111FB7
:104F1000221F331F8A95D2F7C901B8010E94D11F01
:104F20000E94111C81E006C061E070E080E090E02A
:104F3000F5CF80E01F910F91089580E0089580E003
:104F40000895CF93C82F80910203813069F018F043
:104F50008230C9F184C0E0911701F091180180817D
:104F6000823209F07EC007C0E0911701F09118016C
:104F70008081823261F48C2F0E949D27811104C0B0
:104F80008C2F0E94E9261DC081E090E01AC08C2F72
:104F90000E949F27811114C0C43179F048F4CB30AE
:104FA00079F0C03109F061C082E08093020308C04B
:104FB000C93219F0C83321F058C01092020355C00D
:104FC00081E0817054C0C93291F120F5C43179F18A
:104FD000B0F4C73009F047C08EE180931E0182E330
:104FE00080931D018AE080931C0184E180931B0162
:104FF00088E080931A0188E28093190134C0CE5171
:10500000C63088F5EC2FF0E0EA54FE4F80818093A3
:10501000010329C0CE34E9F020F4CB3421F56AE055
:1050200013C0C13579F0C235F1F461E00DC0809153
:105030000103882319F01092010315C081E08093C9
:10504000020315C061E006C0809101030E9423267F
:105050000AC06AE0809101030E94992604C0109260
:10506000020380E004C081E002C080E0AACFCF91BB
:1050700008950E94C923811102C00E94A5230E94A5
:10508000E52380931D0380FF02C0869501C080E068
:105090000C94200380911D03982F9695292F30E0C2
:1050A000233031054CF49F5F990F8170892B81600B
:1050B00080931D030E94E92380911D0386950C9423
:1050C000200380911D03982F969591F09158990F88
:1050D0008170892B80931D038E7F91E009F490E00D
:1050E00080911D0390FB80F980931D030E94E923AA
:1050F00080911D0386950C94200380911D03982FA9
:10510000909590FB80F980931D030E94E923809184
:105110001D0380FF02C0869501C080E00C9420032F
:1051200090911D03892F86958F5F8F7791708430C2
:1051300028F4880F892B80931D0302C090931D03D0
:1051400080911D038E7F91E009F490E080911D0312
:1051500090FB80F980931D030E94E92380911D0339
:1051600086950C94200320911D03922F96958927F4
:10517000982F990F822F8170892B80931D038E7F2A
:1051800091E009F490E080911D0390FB80F98093F9
:105190001D030E94E92380911D0386950C94200332
:1051A00080911D03869508955058BB27AA270ED0DD
:1051B000D1C1C2D130F0C7D120F031F49F3F11F4FA
:1051C0001EF4B7C10EF4E095E7FB9FC1E92FD3D1E0
:1051D00080F3BA17620773078407950718F071F414
:1051E0009EF5EBC10EF4E0950B2EBA2FA02D0B010E
:1051F000B90190010C01CA01A0011124FF27591B1C
:1052000099F0593F50F4503E68F11A16F040A22F21
:10521000232F342F4427585FF3CF46953795279592
:10522000A795F0405395C9F77EF41F16BA0B620B91
:10523000730B840BBAF09150A1F0FF0FBB1F661FD8
:10524000771F881FC2F70EC0BA0F621F731F841F1B
:1052500048F4879577956795B795F7959E3F08F041
:10526000B3CF9395880F08F09927EE0F9795879500
:10527000089527D108F481E008950CD06BC163D163
:1052800040F05AD130F021F45F3F19F03EC1511186
:1052900095C14FC170D198F39923C9F35523B1F348
:1052A000951B550BBB27AA2762177307840738F095
:1052B0009F5F5F4F220F331F441FAA1FA9F333D0F4
:1052C0000E2E3AF0E0E830D091505040E695001CA8
:1052D000CAF729D0FE2F27D0660F771F881FBB1F64
:1052E000261737074807AB07B0E809F0BB0B802D3E
:1052F000BF01FF2793585F4F2AF09E3F510568F08A
:1053000004C15CC15F3FECF3983EDCF38695779572
:105310006795B795F7959F5FC9F7880F911D96958B
:10532000879597F90895E1E0660F771F881FBB1FE7
:10533000621773078407BA0720F0621B730B840B94
:10534000BA0BEE1F88F7E095089504D06894B11168
:1053500035C1089518D188F09F5790F0B92F99273B
:10536000B751A0F0D1F0660F771F881F991F1AF070
:10537000BA95C9F712C0B13081F01FD1B1E00895DC
:105380001CC1672F782F8827B85F39F0B93FCCF35D
:10539000869577956795B395D9F73EF49095809566
:1053A000709561957F4F8F4F9F4F0895E89409C086
:1053B00097FB3EF490958095709561957F4F8F4F48
:1053C0009F4F9923A9F0F92F96E9BB279395F6955E
:1053D000879577956795B795F111F8CFFAF4BB0FDC
:1053E00011F460FF1BC06F5F7F4F8F4F9F4F16C040
:1053F000882311F096E911C0772321F09EE8872FCA
:10540000762F05C0662371F096E8862F70E060E085
:105410002AF09A95660F771F881FDAF7880F9695FE
:10542000879597F9089588D018F011F08CD038F44A
:1054300080C0C4C0E92F9FD0B0F35523C9F3E7FB68
:105440006217730784079507A8F199F3E92FFF27DF
:1054500088232AF03197660F771F881FDAF7952F78
:105460005527442332F091505040220F331F441FE0
:10547000D2F7BB27E91BF50B621B730B840BB10939
:10548000C1F222F4620F731F841FB11D31972AF0FD
:10549000660F771F881FBB1FEFCF915050405AF007
:1054A00041F0882332F0660F771F881F91505040DB
:1054B000C1F7939530C08695779567959F5FD9F72B
:1054C000F8CF990F0008550FAA0BE0E8FEEF16166B
:1054D0001706E807F907C0F012161306E407F507E8
:1054E00098F0621B730B840B950B39F40A2661F05C
:1054F000232B242B252B21F408950A2609F4A140FF
:10550000A6958FEF811D811D089597F99F6780E80B
:1055100070E060E008959F3F31F0915020F487954E
:1055200077956795B795880F911D9695879597F90B
:1055300008959FEF80EC089500240A94161617062C
:1055400018060906089500240A9412161306140674
:1055500005060895092E0394000C11F4882352F0D7
:10556000BB0F40F4BF2B11F460FF04C06F5F7F4F8F
:105570008F4F9F4F089557FD9058440F551F59F076
:105580005F3F71F04795880F97FB991F61F09F3F30
:1055900079F087950895121613061406551FF2CF59
:1055A0004695F1DF08C0161617061806991FF1CFA9
:1055B00086957105610508940895E894BB276627D0
:1055C0007727CB0197F908957CDF08F48FEF0895D2
:1055D0000BD0C0CFB1DF28F0B6DF18F0952309F06B
:1055E00094CFA7CF1124EACFC6DFA0F3959FD1F3C4
:1055F000950F50E0551F629FF001729FBB27F00D81
:10560000B11D639FAA27F00DB11DAA1F649F6627D5
:10561000B00DA11D661F829F2227B00DA11D621F24
:10562000739FB00DA11D621F839FA00D611D221FDE
:10563000749F3327A00D611D231F849F600D211DC2
:10564000822F762F6A2F11249F5750408AF0E1F065
:1056500088234AF0EE0FFF1FBB1F661F771F881FAE
:1056600091505040A9F79E3F510570F04ECFA6CF04
:105670005F3FECF3983EDCF3869577956795B79599
:10568000F795E7959F5FC1F7FE2B880F911D9695C3
:10569000879597F90895FA01EE0FFF1F30962105BF
:1056A000310599F16115710561F48038BFE39B07FD
:1056B00049F168949038810561F08038BFEF9B070D
:1056C00041F0992342F5FF3FE1053105210511F134
:1056D000E8940894E795D901AA2329F4AB2FBE2FAB
:1056E000F85FD0F310C0FF5F70F4A695E0F7F739CC
:1056F00050F019F0FF3A38F49F779F930CD00F9039
:1057000007FC905808953EF014CF60E070E080E808
:105710009FE308954FE79F775F934F933F932F93B6
:105720009ED02F913F914F915F9152DF05C019F4A8
:105730000EF0EBCE42CFFDCE26DFC8F39638C0F791
:1057400007F80F92E8942BE33AEA48EB5FE74EDF65
:105750000F920F920F924DB75EB70F92C0D0EAE052
:10576000F1E016D04F915F91EF91FF91E595EE1F1B
:10577000FF1F49F0FE57E0684427EE0F441FFA95DB
:10578000E1F74195550B32D00F9007FE26C00895E2
:10579000DF93CF931F930F93FF92EF92DF927B01E2
:1057A0008C01689405C0DA2EEF011EDFFE01E8943B
:1057B000A5912591359145915591AEF3EF0106DD07
:1057C000FE019701A801DA9479F7DF90EF90FF903E
:1057D0000F911F91CF91DF9108959B01AC0160E083
:1057E00070E080E89FE349CD90CE95CECCDEE8F323
:1057F0009923D9F3940F511DBBF39150504094F06D
:1058000059F0882332F0660F771F881F915050405F
:10581000C1F79E3F510544F7880F911D96958795D6
:1058200097F908955F3FACF0983E9CF0BB278695B2
:1058300077956795B79508F4B1609395C1F7BB0F5D
:1058400058F711F460FFE8CF6F5F7F4F8F4F9F4F86
:10585000E3CFB4CE0EF05FCE6CCE689456CE93DE1E
:10586000C8F39923D1F3C6F3DF93CF931F930F931C
:10587000FF92C92FDD2788232AF02197660F771F13
:10588000881FDAF720E030E040E85FEB9FE38839DB
:1058900020F0803E30F021968F7787DCE2E3F1E064
:1058A00003C083DCEFE5F1E073DF8B01BE01EC01A7
:1058B000FB2E6F5771097595771F880B990B78DD53
:1058C00028E132E741E35FE38FDEAF2D9801AE01BF
:1058D000FF900F911F91CF91DF9178DC3BCEFA01C1
:1058E000DC01AA0FBB1F9B01AC01BF5728F4222784
:1058F0003327442750781FC0B75188F4AB2F0024BA
:10590000469537952795011CA395D2F3002069F0A1
:10591000220F331F441FB395DAF30DD045CC61300D
:105920007105A0E88A07B94630F49B01AC016627EF
:10593000772788279078309621F02083318342831F
:1059400053830895AA1BBB1B51E107C0AA1FBB1FAD
:10595000A617B70710F0A61BB70B881F991F5A95FB
:10596000A9F780959095BC01CD01089597FB072E6E
:1059700016F4009407D077FD09D00E94A22C07FCF2
:1059800005D03EF4909581959F4F0895709561954F
:105990007F4F0895EE0FFF1F0590F491E02D0994BD
:1059A000F999FECF92BD81BDF89A992780B50895E7
:1059B000A8E1B0E042E050E00C94F82C262FF999D1
:1059C000FECF92BD81BDF89A019700B4021639F05E
:1059D0001FBA20BD0FB6F894FA9AF99A0FBE08952F
:1059E0000196272F0E94DF2C0C94DE2CDC01CB01CA
:1059F000FC01F999FECF06C0F2BDE1BDF89A3196DF
:105A000000B40D9241505040B8F70895F894FFCF7C
:105A1000640007000CFF0000003F643310C1109EBB
:105A2000106A1036100101DF022808140A321E0025
:105A300002040507090B0C0E1011131517181A1C78
:105A40001D1F2123242628292B2D2F3032343537B2
:105A5000393B1F0F03764F5F6F7F496943790959BF
:105A600053633149803F5D8B803FF8BF803FCAE17F
:105A7000803F73ED803FCAE1803FF8BF803F5D8B80
:105A8000803F3149803F0000803FF16D7F3F75EAE4
:105A90007E3F4C827E3F833F7E3F84287E3F833F14
:105AA0007E3F4C827E3F75EA7E3FF16D7F3F000076
:105AB000803F3F4D36394B05FE04C8048F04220455
:105AC0003B0454046D0401020304050607080900A1
:00000001FF
